:1000000007309F0004280000FE308316031385008C
:1000100000308600831203138501FF30860005142B
:10002000851C1428061415280610051D1928861489
:100030001A288610851D1E2886161F288612051E62
:100040002328061724280613051F28280615292803
:100050000611851F2D2886152E2886110510851D51
:100060003328061634280612051E38288617392824
:100070008613051F3D2806153E280611851F4228B8
:080080008615432886110F28A4
:02400E00303F41
:00000001FF
